:020000040800F2
:1000000000060020E1020008E3020008E302000805
:10001000E3020008E3020008E3020008E30200082C
:10002000E3020008E3020008E3020008DD310008F3
:10003000E3020008E3020008E3020008E30200080C
:10004000E3020008E3020008E3020008E3020008FC
:10005000E3020008E3020008C1490008ED49000876
:10006000194A0008454A0008714A0008D5110008DD
:10007000FD1100082912000855120008811200081D
:10008000A9120008D5120008E3020008E3020008E4
:10009000E3020008E3020008E30200089D4A0008AA
:1000A000E3020008E3020008E3020008E30200089C
:1000B000E3020008E3020008E3020008E30200088C
:1000C000E3020008E3020008E3020008E30200087C
:1000D000E3020008754B0008E3020008E302000891
:1000E000014B0008E3020008E3020008E3020008F5
:1000F000E3020008E3020008E3020008011300081D
:10010000E3020008E30200089D4B0008E302000838
:10011000894B0008E3020008E3020008E30200083C
:100120002D1300085513000881130008AD130008B3
:10013000D9130008E3020008E3020008E302000804
:10014000E3020008E3020008E3020008E3020008FB
:10015000011400082D14000859140008E3020008D7
:10016000E3020008E3020008E3020008E3020008DB
:10017000E3020008C93D0008E3020008E3020008AA
:10018000E3020008E3020008E3020008E3020008BB
:10019000E3020008E3020008E3020008E3020008AB
:1001A000E3020008E3020008E3020008E30200089B
:1001B000E3020008E3020008E3020008E30200088B
:1001C000E3020008E3020008E3020008E30200087B
:1001D000E3020008B53D0008E3020008E30200085E
:1001E000E3020008E3020008E3020008E30200085B
:1001F000E3020008E3020008E3020008E30200084B
:10020000E3020008E3020008E3020008E30200083A
:10021000E3020008E3020008E3020008E30200082A
:10022000E3020008E3020008E3020008E30200081A
:10023000E3020008E3020008E3020008E30200080A
:10024000E3020008E3020008E3020008E3020008FA
:10025000E3020008E3020008E3020008E3020008EA
:10026000E3020008E3020008E3020008E3020008DA
:10027000E3020008E3020008E3020008E3020008CA
:10028000E3020008E3020008E3020008E3020008BA
:10029000E3020008E3020008E3020008E3020008AA
:1002A000E3020008E3020008E3020008E30200089A
:1002B000E3020008E3020008E3020008E30200088A
:1002C000E3020008E3020008E3020008E30200087A
:1002D000E3020008E3020008E3020008E30200086A
:1002E00002E000F000F8FEE772B6374880F30888B5
:1002F000364880F3098836483649086040F20000E5
:10030000CCF200004EF63471CEF200010860BFF36B
:100310004F8FBFF36F8F40F20000C0F2F0004EF637
:100320008851CEF200010860BFF34F8FBFF36F8F8B
:100330004FF00000E1EE100A4EF63C71CEF20001E3
:100340000860062080F31488BFF36F8F02F0A8FFC7
:1003500004F0F0F84FF055301F491B4A91423CBF62
:1003600041F8040BFAE71D49184A91423CBF41F895
:10037000040BFAE71A491B4A1B4B9A423EBF51F83D
:10038000040B42F8040BF8E700201849184A914280
:100390003CBF41F8040BFAE702F0C0FF04F04EF94D
:1003A000144C154DAC4203DA54F8041B8847F9E7A6
:1003B00000F042F8114C124DAC4203DA54F8041B21
:1003C0008847F9E702F0A8BF0006002000220020BD
:1003D0000000000808ED00E00000002000060020FA
:1003E000105100080022002068220020682200200E
:1003F0007C4D0020E0020008E0020008E002000856
:10040000E00200082DE9F04F2DED108AC1F80CD064
:10041000D0F80CD0BDEC108ABDE8F08F002383F338
:1004200011882846A047002002F090F9FEE702F06C
:100430001BF900DFFEE7000038B500F0D3FC00F048
:10044000A1FE02F08BFE054602F0BEFE0446C0B9D6
:100450000E4B9D4217D001339D4241F2883512BFA9
:10046000044600250124002002F082FE0CB100F0B9
:1004700075F800F027FE284600F01EF900F06EF82F
:10048000F9E70025EFE70546EDE700BF010007B0FB
:1004900008B500F073FCA0F120035842584108BD94
:1004A00007B541F21203022101A8ADF8043000F0B3
:1004B00083FC03B05DF804FB38B5302383F3118867
:1004C000174803680BB102F00DFA0023154A4FF4E8
:1004D0007A71134802F0FCF9002383F31188124C5F
:1004E000236813B12368013B2360636813B1636819
:1004F000013B63600D4D2B7833B963687BB90220F3
:1005000000F042FD322363602B78032B07D1636830
:100510002BB9022000F038FD4FF47A73636038BDC8
:1005200068220020B90400088823002080220020CF
:10053000084B187003280CD8DFE800F00805020803
:10054000022000F011BD022000F000BD024B00228D
:100550005A6070478022002088230020F8B5504B55
:10056000504A1C461968013100F0998004339342C7
:10057000F8D162684C4B9A4240F291804B4B9B6899
:1005800003F1006303F500339A4280F08880002075
:1005900000F04EFC0220FFF7CBFF454B0021D3F8C3
:1005A000E820C3F8E810D3F81021C3F81011D3F8ED
:1005B0001021D3F8EC20C3F8EC10D3F81421C3F8C1
:1005C0001411D3F81421D3F8F020C3F8F010D3F8A5
:1005D0001821C3F81811D3F81821D3F8802042F05D
:1005E0000062C3F88020D3F8802022F00062C3F8B4
:1005F0008020D3F88020D3F8802042F00072C3F826
:100600008020D3F8802022F00072C3F88020D3F835
:10061000803072B64FF0E023C3F8084DD4E90004EF
:10062000BFF34F8FBFF36F8F224AC2F88410BFF31E
:100630004F8F536923F480335361BFF34F8FD2F848
:10064000803043F6E076C3F3C905C3F34E335B0154
:1006500003EA060C29464CEA81770139C2F8747224
:10066000F9D2203B13F1200FF2D1BFF34F8FBFF32C
:100670006F8FBFF34F8FBFF36F8F536923F4003336
:1006800053610023C2F85032BFF34F8FBFF36F8F17
:10069000302383F31188854680F308882047F8BD0E
:1006A0000000020820000208FFFF010800220020CD
:1006B0000044025800ED00E02DE9F04F93B0B44B38
:1006C0002022FF2100900AA89D6800F0A5FCB14AF5
:1006D0001378A3B90121B04811700360302383F36C
:1006E000118803680BB102F0FDF80023AB4A4FF408
:1006F0007A71A94802F0ECF8002383F31188009B7B
:1007000013B1A74B009A1A60A64A1378032B03D0A3
:1007100000231370A24A53604FF0000A009CD34696
:100720005646D146012000F01FFC24B19C4B1B68AB
:10073000002B00F02682002000F020FB0390039B9A
:10074000002BF2DB012000F001FC039B213B1F2B5F
:10075000E8D801A252F823F0D907000801080008E0
:100760009508000825070008250700082507000848
:1007700027090008F70A0008110A0008730A000890
:100780009B0A0008C10A000825070008D30A0008D0
:1007900025070008450B0008790800082507000810
:1007A000890B0008E50700087908000825070008FC
:1007B000730A000825070008250700082507000818
:1007C0002507000825070008250700082507000859
:1007D00025070008950800080220FFF759FE0028A9
:1007E00040F0F981009B022105A8BAF1000F08BF73
:1007F0001C4641F21233ADF8143000F0DDFA91E7F7
:100800004FF47A7000F0BAFA071EEBDB0220FFF714
:100810003FFE0028E6D0013F052F00F2DE81DFE831
:1008200007F0030A0D1013360523042105A80593CC
:1008300000F0C2FA17E004215548F9E704215A48AC
:10084000F6E704215948F3E74FF01C08404608F149
:10085000040800F0EFFA0421059005A800F0ACFAB6
:10086000B8F12C0FF2D101204FF0000900FA07F780
:1008700047EA0B0B5FFA8BFB00F01AFC26B10BF07A
:100880000B030B2B08BF0024FFF70AFE4AE70421E5
:100890004748CDE7002EA5D00BF00B030B2BA1D1C1
:1008A0000220FFF7F5FD074600289BD00120002617
:1008B00000F0BEFA0220FFF73BFE1FFA86F8404622
:1008C00000F0C6FA0446B0B1039940460136A1F1E2
:1008D00040025142514100F0CBFA0028EDD1BA4616
:1008E000044641F21213022105A83E46ADF8143029
:1008F00000F062FA16E725460120FFF719FE244BA7
:100900009B68AB4207D9284600F094FA013040F0CA
:1009100067810435F3E70025224BBA463E461D7039
:100920001F4B5D60A8E7002E3FF45CAF0BF00B039C
:100930000B2B7FF457AF0220FFF7FAFD322000F0B7
:100940001DFAB0F10008FFF64DAF18F003077FF471
:1009500049AF0F4A08EB0503926893423FF642AF56
:10096000B8F5807F3FF73EAF124BB845019323DDCA
:100970004FF47A7000F002FA0390039A002AFFF60F
:1009800031AF039A0137019B03F8012BEDE700BF5C
:10099000002200208423002068220020B9040008DF
:1009A000882300208022002004220020082200202A
:1009B0000C22002084220020C820FFF769FD074692
:1009C00000283FF40FAF1F2D11D8C5F120020AAB4C
:1009D00025F0030084494245184428BF424601924D
:1009E00000F0F4FA019AFF217F4800F015FB4FEA6E
:1009F000A803C8F387027C492846019300F014FB42
:100A0000064600283FF46DAF019B05EB830533E7F5
:100A10000220FFF73DFD00283FF4E4AE00F046FA67
:100A200000283FF4DFAE0027B846704B9B68BB42FE
:100A300018D91F2F11D80A9B01330ED027F00303BA
:100A400012AA134453F8203C05934046042205A9FA
:100A5000043700F0A9FB8046E7E7384600F0EAF9E2
:100A60000590F2E7CDF81480042105A800F0A4F960
:100A700002E70023642104A8049300F093F90028FE
:100A80007FF4B0AE0220FFF703FD00283FF4AAAECA
:100A9000049800F001FA0590E6E70023642104A819
:100AA000049300F07FF900287FF49CAE0220FFF74A
:100AB000EFFC00283FF496AE049800F0EFF9EAE767
:100AC0000220FFF7E5FC00283FF48CAE00F0FEF9B1
:100AD000E1E70220FFF7DCFC00283FF483AE05A924
:100AE000142000F0F9F907460421049004A800F04E
:100AF00063F93946B9E7322000F040F9071EFFF6E6
:100B000071AEBB077FF46EAE384A07EB09039268FB
:100B100093423FF667AE0220FFF7BAFC00283FF48D
:100B200061AE27F003074F44B9453FF4A5AE4846F0
:100B300009F1040900F07EF90421059005A800F0F0
:100B40003BF9F1E74FF47A70FFF7A2FC00283FF47D
:100B500049AE00F0ABF9002844D00A9B01330BD01A
:100B600008220AA9002000F05FFA00283AD02022CB
:100B7000FF210AA800F050FAFFF792FC1C4801F090
:100B8000EBFD13B0BDE8F08F002E3FF42BAE0BF061
:100B90000B030B2B7FF426AE0023642105A80593DD
:100BA00000F000F9074600287FF41CAE0220FFF792
:100BB0006FFC804600283FF415AEFFF771FC41F250
:100BC000883001F0C9FD059800F0BAFA46463C4667
:100BD00000F06EFAA6E506464EE64FF0000901E683
:100BE000BA467EE637467CE68422002000220020BA
:100BF000A08601002DE9F84F4FF47A7306460D46A2
:100C0000002402FB03F7DFF85080DFF8509098F9DA
:100C100000305FFA84FA5A1C01D0A34210D159F86F
:100C200024002A4631460368D3F820B03B46D84713
:100C3000854205D1074B012083F800A0BDE8F88F5D
:100C40000134032CE3D14FF4FA7001F085FD00204C
:100C5000F4E700BFD423002010220020142200203B
:100C600000232DE9F0471A4605468846012019461B
:100C700000F09AFC0446802002F000FA07460028A3
:100C800061D0002C5FD03B4E28464FF0800A73693C
:100C900043F0C0637361D6F8143143F0C063C6F803
:100CA000143102F06FF805EB080200FB05F34FF476
:100CB000D06C50434FF03D0E834233D23269520123
:100CC00043D4D6F8102151013FD4216803F10062CA
:100CD0008A602268D7602268C2F804A02268C2F83D
:100CE00000C0D4F80090D9F8002042F00102C9F801
:100CF0000020D4F80090D9F8002022F01E02C9F894
:100D00000020D4F80090D9F80020D207FBD494F842
:100D10000C90803361680EFA09F20A60CCE700207B
:100D200002F00EF9204600F07FFC384602F0DCF9B4
:100D3000104B5A6942F0C0625A61D3F8142142F054
:100D4000C062C3F81421BDE8F0870B4B9A6A42F4E5
:100D500000729A629A6A42F400429A6261B6002670
:100D6000012002F0EDF8B045D9D9A819013602F0FA
:100D700021F8F8E70020005200ED00E0002307B55D
:100D8000024601210DF107008DF80730FFF732FF11
:100D900020B19DF8070003B05DF804FB4FF0FF3071
:100DA000F9E700000A46042108B5FFF723FF80F0A9
:100DB0000100C0B2404208BD074B0A4630B4197862
:100DC000064B53F82140014623682046DD69044B59
:100DD000AC4630BC604700BFD42300201422002062
:100DE000A086010070B5104C0025104E01F0CEFF1A
:100DF00020803068238883420CD800252088013861
:100E000001F0C0FF23880544013BB5F5802F238006
:100E1000F4D370BD01F0B6FF336805440133B5F576
:100E2000003F3360E5D3E8E7D6230020902300207D
:100E300002F086B800F1006000F5003000687047ED
:100E400000F10060920000F5003001F0FBBF0000EF
:100E5000054B1A68054B1B889B1A834202D9104424
:100E600001F090BF0020704790230020D62300207F
:100E700038B50446074D29B128682044BDE83840FC
:100E800001F098BF2868204401F082FF0028F3D0C9
:100E900038BD00BF902300200020704700F1FF50B4
:100EA00000F58F10D0F8000870470000064991F84F
:100EB000243033B100230822086A81F82430FFF778
:100EC000BFBF0120704700BF94230020014B18686A
:100ED000704700BF0010005C194B01380322084422
:100EE00070B51D68174BC5F30B042D0C1E88A64268
:100EF0000BD15C680A46013C824213460FD214F9BA
:100F0000016F4EB102F8016BF6E7013A03F10803F5
:100F1000ECD181420B4602D22C2203F8012B04248F
:100F2000094A1688AE4204D1984284BF967803F8E5
:100F3000016B013C02F10402F3D1581A70BD00BFED
:100F40000010005C20220020A84C0008022803D1D9
:100F5000044B10229A6170470128FCD1014B2022DA
:100F6000F8E700BF00100258022804D1054B4FF4E7
:100F700080129A6170470128FCD1024B4FF4001295
:100F8000F7E700BF00100258022805D1064A53694E
:100F900083F01003536170470128FCD1024A536962
:100FA00083F02003F6E700BF0010025870B5044636
:100FB0004FF47A764CB1412C254628BF412506FBDB
:100FC00005F0641B01F0C8FBF4E770BD002310B509
:100FD000934203D0CC5CC4540133F9E710BD000048
:100FE000013810B510F9013F3BB191F900409C4226
:100FF00003D11AB10131013AF4E71AB191F9002095
:10100000981A10BD1046FCE703460246D01A12F9A2
:10101000011B0029FAD1704702440346934202D0D3
:1010200003F8011BFAE770472DE9F8431F4D1446FA
:101030000746884695F8242052BBDFF870909CB391
:1010400095F824302BB92022FF2148462F62FFF764
:10105000E3FF95F824004146C0F1080205EB80004B
:10106000A24228BF2246D6B29200FFF7AFFF95F802
:101070002430A41B17441E449044E4B2F6B2082E58
:1010800085F82460DBD1FFF711FF0028D7D108E0F5
:101090002B6A03EB82038342CFD0FFF707FF0028C0
:1010A000CBD10020BDE8F8830120FBE7942300208A
:1010B000024B1A78024B1A70704700BFD4230020ED
:1010C00010220020F8B5194C194800F075FE214691
:1010D000174800F09DFE24684FF47A70154ED4F83E
:1010E0009020154DD2F80438114F43F00203C2F896
:1010F0000438FFF75BFF2046104900F097FFD4F853
:1011000090200324D2F8043823F00203C2F80438F4
:101110004FF4E133336055F8040BB84202D0314646
:1011200000F0A8FD013CF6D1F8BD00BFA44E0008B8
:10113000A82F0020BC23002014220020AC4E000861
:101140000C4B70B50C4D04461E780C4B55F8262000
:101150009A420DD00A4B002118221846FFF75CFF77
:101160000460014655F82600BDE8704000F082BDDD
:1011700070BD00BFD423002014220020A82F00201F
:10118000BC23002008B571B6054B1988054B18889B
:10119000FFF766FD02210E20FFF762FD61B608BD74
:1011A000D62300209023002030B50A44084D9142F8
:1011B0000DD011F8013B5840082340F30004013BD7
:1011C0002C4013F0FF0384EA5000F6D1EFE730BD66
:1011D0002083B8ED08B5074B074A196801F03D01B7
:1011E000996053680BB190689847BDE8084002F0D9
:1011F0002DB800BF00000240D823002008B5084BDE
:101200001968890901F03D018A019A60054AD3688D
:101210000BB110699847BDE8084002F017B800BF4D
:1012200000000240D823002008B5084B1968090CBB
:1012300001F03D010A049A60054A53690BB19069B7
:101240009847BDE8084002F001B800BF0000024026
:10125000D823002008B5084B1968890D01F03D011D
:101260008A059A60054AD3690BB1106A9847BDE8B0
:10127000084001F0EBBF00BF00000240D82300206F
:1012800008B5074B074A596801F03D01D960536A18
:101290000BB1906A9847BDE8084001F0D7BF00BF86
:1012A00000000240D823002008B5084B596889097E
:1012B00001F03D018A01DA60054AD36A0BB1106B77
:1012C0009847BDE8084001F0C1BF00BF00000240E0
:1012D000D823002008B5084B5968090C01F03D01DE
:1012E0000A04DA60054A536B0BB1906B9847BDE86E
:1012F000084001F0ABBF00BF00000240D82300202F
:1013000008B5084B5968890D01F03D018A05DA607E
:10131000054AD36B0BB1106C9847BDE8084001F04B
:1013200095BF00BF00000240D823002008B5074B3E
:10133000074A196801F03D019960536C0BB1906C3C
:101340009847BDE8084001F081BF00BF000402409B
:10135000D823002008B5084B1968890901F03D0120
:101360008A019A60054AD36C0BB1106D9847BDE8AD
:10137000084001F06BBF00BF00040240D8230020EA
:1013800008B5084B1968090C01F03D010A049A6080
:10139000054A536D0BB1906D9847BDE8084001F0C8
:1013A00055BF00BF00040240D823002008B5084BF9
:1013B0001968890D01F03D018A059A60054AD36DCF
:1013C0000BB1106E9847BDE8084001F03FBF00BF69
:1013D00000040240D823002008B5074B074A59688B
:1013E00001F03D01D960536E0BB1906E9847BDE896
:1013F000084001F02BBF00BF00040240D8230020AA
:1014000008B5084B5968890901F03D018A01DA6085
:10141000054AD36E0BB1106F9847BDE8084001F044
:1014200015BF00BF00040240D823002008B5084BB8
:101430005968090C01F03D010A04DA60054A536F4E
:101440000BB1906F9847BDE8084001F0FFBE00BFA8
:1014500000040240D823002008B5084B5968890DC4
:1014600001F03D018A05DA60054AD36F13B1D2F865
:1014700080009847BDE8084001F0E8BE0004024043
:10148000D823002000230C4910B51A460B4C0B60E2
:1014900054F82300026001EB430004334260402B08
:1014A000F6D1074A4FF0FF339360D360C2F8083497
:1014B000C2F80C3410BD00BFD8230020B84C00087F
:1014C000000002400F28F8B510D9102810D01128BC
:1014D00011D0122808D10F240720DFF8C8E0012618
:1014E000DEF80050A04208D9002653E00446F4E795
:1014F0000F240020F1E70724FBE706FA00F73D423E
:101500004AD1264C4FEA001C3D4304EB00160EEB7B
:10151000C000CEF80050C0E90123FBB273B12048EF
:10152000D0F8D83043F00103C0F8D830D0F80031FB
:1015300043F00103C0F80031D0F8003117F47F4FB9
:101540000ED01748D0F8D83043F00203C0F8D83096
:10155000D0F8003143F00203C0F80031D0F8003178
:1015600054F80C00036823F01F030360056815F0AE
:101570000105FBD104EB0C033D2493F80CC05F681C
:1015800004FA0CF43C6021240560446112B1987B9C
:1015900000F0A4F93046F8BD0130A3E7B84C0008CC
:1015A00000440258D823002010B5302484F3118859
:1015B000FFF788FF002383F3118810BD10B50446A0
:1015C000807B00F0A1F901231549627B03FA02F246
:1015D0000B6823EA0203DAB20B6072B9114AD2F83F
:1015E000D81021F00101C2F8D810D2F8001121F072
:1015F0000101C2F80011D2F8002113F47F4F0ED17F
:10160000084BD3F8D82022F00202C3F8D820D3F830
:10161000002122F00202C3F80021D3F8003110BDEE
:10162000D82300200044025808B5302383F31188E2
:10163000FFF7C4FF002383F3118808BD02684368E5
:101640001143016003B1184770470000024A136854
:1016500043F0C0031360704700100140024A136852
:1016600043F0C00313607047004C004037B51A4C7C
:101670001A4D204600F0F2FA04F114000094002301
:101680004FF40072164900F0AFF94FF4007215499B
:1016900004F138000094144B00F028FA134BC4E90D
:1016A0001735134C204600F0D9FA04F1140000233A
:1016B0004FF400720F49009400F096F90E4B4FF46E
:1016C00000720E4904F13800009400F00FFA0C4B40
:1016D000C4E9173503B030BD5C24002000E1F505F6
:1016E00034250020342900204D1600080010014048
:1016F000C8240020342700205D160008342B002069
:10170000004C0040037C30B52D4C002918BF0C461E
:10171000012B11D12B4B98423BD12B4BD3F8F0200E
:1017200042F01002C3F8F020D3F8182142F0100262
:10173000C3F81821D3F818312268036EC16D03EB8A
:1017400052038466B3FBF2F36268150442BF23F0D0
:10175000070503F0070343EA4503CB60A36843F0A2
:1017600040034B60E36843F001038B6042F49673DF
:1017700043F001030B604FF0FF330B62510505D5B9
:1017800012F0102218D0B2F1805F17D080F86430C8
:1017900030BD0E4B9842CFD10B4BD3F8E82042F42A
:1017A0000022C3F8E820D3F8102142F40022C3F845
:1017B0001021D3F81031BFE77F23E7E73F23E5E7A8
:1017C000B84D00085C24002000440258C8240020C2
:1017D0002DE9F047C66D05463768F4692107346284
:1017E0001AD014F0080118BF4FF48071E20748BF07
:1017F00041F02001A3074FF0300348BF41F0400102
:10180000600748BF41F0800183F31188281DFFF76E
:1018100015FF002383F31188E2050AD5302383F3F3
:1018200011884FF48061281DFFF708FF002383F320
:1018300011884FF030094FF0000A14F0200838D119
:101840003B0616D54FF0300905F1380A200610D5B1
:1018500089F31188504600F07DF9002836DA082116
:10186000281DFFF7EBFE27F080033360002383F38E
:101870001188790614D5620612D5302383F31188B6
:10188000D5E913239A4208D12B6C33B127F04007D6
:101890001021281DFFF7D2FE3760002383F3118843
:1018A000E30618D5AA6E1369ABB15069BDE8F047DD
:1018B000184789F31188736A284695F8641019400F
:1018C00000F0E6F98AF31188F469B6E7B06288F3AC
:1018D0001188F469BAE7BDE8F0870000090100F15A
:1018E0006043012203F56143C9B283F8001300F09D
:1018F0001F039A4043099B0003F1604303F56143D2
:10190000C3F880211A60704700F01F0301229A403B
:10191000430900F160409B0000F5614003F1604322
:1019200003F56143C3F88020C3F88021002380F8C9
:1019300000337047F8B51546826804460B46AA4244
:1019400000D28568A1692669761AB5420BD218467D
:101950002A46FFF73BFBA3692B44A3612846A368F3
:101960005B1BA360F8BD0CD9AF1B18463246FFF7CE
:101970002DFB3A46E1683044FFF728FBE3683B441F
:10198000EBE718462A46FFF721FBE368E5E700008E
:1019900083689342F7B50446154600D28568D4E9BA
:1019A0000460361AB5420BD22A46FFF70FFB636973
:1019B0002B4463612846A3685B1BA36003B0F0BDA2
:1019C0000DD93246AF1B0191FFF700FB01993A4652
:1019D000E0683144FFF7FAFAE3683B44E9E72A4656
:1019E000FFF7F4FAE368E4E710B50A440024C361A2
:1019F000029B8460C16002610362C0E90000C0E92B
:101A0000051110BD08B5D0E90532934201D18268B5
:101A100082B98268013282605A1C426119700021C9
:101A2000D0E904329A4224BFC368436100F0B0FE9B
:101A3000002008BD4FF0FF30FBE7000070B53023F9
:101A400004460E4683F31188A568A5B1A368A26970
:101A5000013BA360531CA36115782269934224BF04
:101A6000E368A361E3690BB120469847002383F341
:101A70001188284607E03146204600F079FE00280C
:101A8000E2DA85F3118870BD2DE9F74F04460E4662
:101A900017469846D0F81C904FF0300A8AF3118808
:101AA0004FF0000B154665B12A4631462046FFF738
:101AB00041FF034660B94146204600F059FE002828
:101AC000F1D0002383F31188781B03B0BDE8F08FB9
:101AD000B9F1000F03D001902046C847019B8BF35A
:101AE0001188ED1A1E448AF31188DCE7C160C361D6
:101AF000009B82600362C0E905111144C0E9000047
:101B000001617047F8B504460D461646302383F34D
:101B10001188A768A7B1A368013BA36063695A1C39
:101B200062611D70D4E904329A4224BFE3686361A4
:101B3000E3690BB120469847002080F3118807E045
:101B40003146204600F014FE0028E2DA87F31188BF
:101B5000F8BD0000D0E9052310B59A4201D1826892
:101B60007AB982680021013282605A1C82611C7835
:101B700003699A4224BFC368836100F009FE2046CE
:101B800010BD4FF0FF30FBE72DE9F74F04460E463E
:101B900017469846D0F81C904FF0300A8AF3118807
:101BA0004FF0000B154665B12A4631462046FFF737
:101BB000EFFE034660B94146204600F0D9FD0028FB
:101BC000F1D0002383F31188781B03B0BDE8F08FB8
:101BD000B9F1000F03D001902046C847019B8BF359
:101BE0001188ED1A1E448AF31188DCE70268436805
:101BF0001143016003B11847704700001430FFF72C
:101C000043BF00004FF0FF331430FFF73DBF00002B
:101C10003830FFF7B9BF00004FF0FF333830FFF71F
:101C2000B3BF00001430FFF709BF00004FF0FF31D1
:101C30001430FFF703BF00003830FFF763BF000028
:101C40004FF0FF323830FFF75DBF0000012914BFAD
:101C50006FF0130000207047FFF708BD044B0360CE
:101C600000234360C0E9023301230374704700BFBF
:101C7000D04D000810B53023044683F31188FFF7D8
:101C800041FD02230020237480F3118810BD000061
:101C900038B5C36904460D461BB904210844FFF753
:101CA000A5FF294604F11400FFF7ACFE002806DA70
:101CB000201D4FF40061BDE83840FFF797BF38BDE5
:101CC000026843681143016003B118477047000080
:101CD00013B5406B00F58054D4F8A4381A68117815
:101CE000042914D1017C022911D119790123128907
:101CF0008B4013420BD101A94C3002F097F9D4F874
:101D0000A4480246019B2179206800F0DFF902B067
:101D100010BD0000143002F019B900004FF0FF337D
:101D2000143002F013B900004C3002F0EBB900009F
:101D30004FF0FF334C3002F0E5B90000143002F0F0
:101D4000E7B800004FF0FF31143002F0E1B80000B6
:101D50004C3002F0B7B900004FF0FF324C3002F0C7
:101D6000B1B900000020704710B500F58054D4F8D8
:101D7000A4381A681178042917D1017C022914D1DA
:101D80005979012352898B4013420ED1143002F04D
:101D900079F8024648B1D4F8A4484FF44073617909
:101DA0002068BDE8104000F07FB910BD406BFFF720
:101DB000DBBF0000704700007FB5124B01250426F1
:101DC000044603600023057400F184024360294641
:101DD000C0E902330C4B0290143001934FF440736E
:101DE000009602F02BF8094B04F69442294604F1C0
:101DF0004C000294CDE900634FF4407302F0F2F816
:101E000004B070BDF84D0008AD1D0008D11C0008DD
:101E10000A68302383F311880B790B3342F82300CF
:101E20004B79133342F823008B7913B10B3342F80B
:101E3000230000F58053C3F8A41802230374002084
:101E400080F311887047000038B5037F044613B152
:101E500090F85430ABB90125201D0221FFF730FF67
:101E600004F114006FF00101257700F09DFC04F1EE
:101E70004C0084F854506FF00101BDE8384000F088
:101E800093BC38BD10B5012104460430FFF718FF9C
:101E90000023237784F8543010BD000038B5044681
:101EA0000025143001F0E2FF04F14C00257702F028
:101EB000B1F8201D84F854500121FFF701FF20469E
:101EC000BDE83840FFF750BF90F8803003F0600362
:101ED000202B06D190F881200023212A03D81F2A25
:101EE00006D800207047222AFBD1C0E91D3303E049
:101EF000034A426707228267C3670120704700BF19
:101F00003822002037B500F58055D5F8A4381A6876
:101F1000117804291AD1017C022917D119790123DA
:101F200012898B40134211D100F14C04204602F07B
:101F300031F958B101A9204602F078F8D5F8A44843
:101F40000246019B2179206800F0C0F803B030BD43
:101F500001F10B03F0B550F8236085B004460D463F
:101F6000FEB1302383F3118804EB8507301D08216F
:101F7000FFF7A6FEFB6806F14C005B691B681BB10E
:101F8000019002F061F8019803A902F04FF80246AF
:101F900048B1039B2946204600F098F8002383F3BC
:101FA000118805B0F0BDFB685A691268002AF5D0A7
:101FB0001B8A013B1340F1D104F18002EAE70000E3
:101FC000133138B550F82140ECB1302383F3118838
:101FD00004F58053D3F8A4281368527903EB8203E5
:101FE000DB689B695D6845B104216018FFF768FEF6
:101FF000294604F1140001F04FFF2046FFF7B4FE1C
:10200000002383F3118838BD7047000001F01CBA2B
:1020100001234022002110B5044600F8303BFEF7B2
:10202000FBFF0023C4E9013310BD000010B53023CD
:10203000044683F311882422416000210C30FEF70E
:10204000EBFF204601F022FA02230020237080F3E8
:10205000118810BD70B500EB8103054650690E462E
:102060001446DA6018B110220021FEF7D5FFA069EE
:1020700018B110220021FEF7CFFF31462846BDE8F7
:10208000704001F009BB000083682022002103F0AA
:10209000011310B5044683601030FEF7BDFF2046E3
:1020A000BDE8104001F084BBF0B4012500EB8104D1
:1020B00047898D40E4683D43A4694581236000233E
:1020C000A2606360F0BC01F0A1BB0000F0B4012588
:1020D00000EB810407898D40E4683D436469058114
:1020E00023600023A2606360F0BC01F017BC000015
:1020F00070B5022300250446242203702946C0F847
:1021000088500C3040F8045CFEF786FF204684F8C7
:10211000705001F055FA63681B6823B129462046C8
:10212000BDE87040184770BD0378052B10B5044614
:102130000AD080F88C300523037043681B680BB10C
:10214000042198470023A36010BD000001780529F1
:1021500006D190F88C20436802701B6803B11847C1
:102160007047000070B590F87030044613B100233A
:1021700080F8703004F18002204601F03DFB636876
:102180009B68B3B994F8803013F0600535D0002116
:10219000204601F02FFE0021204601F01FFE63685B
:1021A0001B6813B1062120469847062384F8703037
:1021B00070BD204698470028E4D0B4F88630A26F5E
:1021C0009A4288BFA36794F98030A56F002B4FF027
:1021D000300380F20381002D00F0F280092284F8A0
:1021E000702083F3118800212046D4E91D23FFF7D6
:1021F0006DFF002383F31188DAE794F8812003F060
:102200007F0343EA022340F20232934200F0C5808A
:1022100021D8B3F5807F48D00DD8012B3FD0022BB9
:1022200000F09380002BB2D104F188026267022291
:10223000A267E367C1E7B3F5817F00F09B80B3F548
:10224000407FA4D194F88230012BA0D1B4F888301B
:1022500043F0020332E0B3F5006F4DD017D8B3F569
:10226000A06F31D0A3F5C063012B90D863682046DE
:1022700094F882205E6894F88310B4F88430B047F4
:10228000002884D0436863670368A3671AE0B3F546
:10229000106F36D040F6024293427FF478AF5C4B29
:1022A00063670223A3670023C3E794F88230012BFE
:1022B0007FF46DAFB4F8883023F00203A4F88830BF
:1022C000C4E91D55E56778E7B4F88030B3F5A06F31
:1022D0000ED194F88230204684F88A3001F0CEF98D
:1022E00063681B6813B101212046984703232370BC
:1022F0000023C4E91D339CE704F18B0363670123CA
:10230000C3E72378042B10D1302383F311882046B0
:10231000FFF7BAFE85F311880321636884F88B50B8
:1023200021701B680BB12046984794F88230002B2F
:10233000DED084F88B300423237063681B68002B85
:10234000D6D0022120469847D2E794F88430204620
:102350001D0603F00F010AD501F040FA012804D050
:1023600002287FF414AF2B4B9AE72B4B98E701F030
:1023700027FAF3E794F88230002B7FF408AF94F843
:10238000843013F00F01B3D01A06204602D501F0B5
:1023900049FDADE701F03AFDAAE794F88230002B41
:1023A0007FF4F5AE94F8843013F00F01A0D01B0633
:1023B000204602D501F01EFD9AE701F00FFD97E7D8
:1023C000142284F8702083F311882B462A4629466C
:1023D0002046FFF769FE85F31188E9E65DB1152215
:1023E00084F8702083F3118800212046D4E91D234E
:1023F000FFF75AFEFDE60B2284F8702083F3118864
:102400002B462A4629462046FFF760FEE3E700BF39
:10241000284E0008204E0008244E000838B590F8D9
:1024200070300446002B3ED0063BDAB20F2A34D877
:102430000F2B32D8DFE803F0373131082232313147
:102440003131313131313737856FB0F886309D42C7
:1024500014D2C3681B8AB5FBF3F203FB12556DB9A6
:10246000302383F311882B462A462946FFF72EFE98
:1024700085F311880A2384F870300EE0142384F861
:102480007030302383F31188002320461A46194602
:10249000FFF70AFE002383F3118838BDC36F03B131
:1024A00098470023E7E70021204601F0A3FC002124
:1024B000204601F093FC63681B6813B10621204697
:1024C00098470623D7E7000010B590F8703004460F
:1024D000142B29D017D8062B05D001D81BB110BD5D
:1024E000093B022BFBD80021204601F083FC002190
:1024F000204601F073FC63681B6813B10621204677
:102500009847062319E0152BE9D10B2380F870308A
:10251000302383F3118800231A461946FFF7D6FDAE
:10252000002383F31188DAE7C3689B695B68002B9B
:10253000D5D1C36F03B19847002384F87030CEE73C
:1025400000238268037503691B6899689142FBD276
:102550005A680360426010605860704700238268C8
:10256000037503691B6899689142FBD85A68036038
:10257000426010605860704708B50846302383F306
:1025800011880A7D0023052A06D8DFE802F00B0532
:102590000503120E826913604FF0FF338361FFF76A
:1025A000CFFF002383F3118808BD8269936801334C
:1025B0009360D0E9003213605A60EDE7FFF7C0BFC7
:1025C000054BD96808751868026853601A600122C3
:1025D000D8600275FDF716BF382D00200C4B30B5C2
:1025E000DD684B1C87B004460FD02B46094A68466D
:1025F00000F06EF92046FFF7E3FF009B13B1684639
:1026000000F070F9A86907B030BDFFF7D9FFF9E70E
:10261000382D00207925000838B50C4D044681611D
:10262000EB6881689A68914203D8BDE83840FFF7AB
:1026300087BF1846FFF792FF01230146EC60204652
:102640002375BDE83840FDF7DDBE00BF382D002002
:10265000044B1A68DB6890689B68984294BF00201E
:1026600001207047382D0020084B10B51C68D86831
:10267000226853601A600122DC602275FFF76EFF4A
:1026800001462046BDE81040FDF7BCBE382D0020B5
:1026900038B50123084C00252370656001F0B6FDB4
:1026A00001F0DCFD0549064801F0B0FE022323706D
:1026B00085F3118838BD00BFA02F0020304E0008E0
:1026C000382D002000F044B9034A516853685B1A62
:1026D0009842FBD8704700BF001000E08B600223D7
:1026E000086108468B8270478368A3F1840243F82F
:1026F000142C026943F8442C426943F8402C094ADF
:1027000043F8242CC268A3F1200043F8182C0222BD
:1027100003F80C2C002203F80B2C034A43F8102C6E
:10272000704700BF1D040008382D002008B5FFF7D2
:10273000DBFFBDE80840FFF741BF0000024BDB684C
:1027400098610F20FFF73CBF382D0020302383F322
:102750001188FFF7F3BF000008B50146302383F36B
:1027600011880820FFF73AFF002383F3118808BD82
:10277000064BDB6839B1426818605A6013604360E9
:102780000420FFF72BBF4FF0FF307047382D00209B
:102790000368984206D01A68026050601846996132
:1027A000FFF70CBF7047000038B504460D4620689F
:1027B000844200D138BD036823605C608561FFF707
:1027C000FDFEF4E7036810B59C68A2420CD85C6873
:1027D0008A600B604C602160596099688A1A9A601F
:1027E0004FF0FF33836010BD121B1B68ECE7000045
:1027F0000A2938BF0A2170B504460D460A26601919
:1028000001F0FEFC01F0E6FC041BA54203D8751C98
:1028100004462E46F3E70A2E04D90120BDE8704095
:1028200001F034BE70BD0000F8B5144B0D460A2A05
:102830004FF00A07D96103F11001826038BF0A2204
:10284000416019691446016048601861A81801F0D8
:10285000C7FC01F0BFFC431B0646A34206D37C1C09
:1028600028192746354601F0CBFCF2E70A2F04D998
:102870000120BDE8F84001F009BEF8BD382D002068
:10288000F8B506460D4601F0A5FC0F4A134653F86D
:10289000107F9F4206D12A4601463046BDE8F840E7
:1028A000FFF7C2BFD169BB68441A2C1928BF2C4658
:1028B000A34202D92946FFF79BFF2246314603482F
:1028C000BDE8F840FFF77EBF382D0020482D0020DE
:1028D000C0E90323002310B45DF8044B4361FFF704
:1028E000CFBF000010B5194C236998420DD0816804
:1028F000D0E9003213605A609A680A449A60002353
:1029000003604FF0FF33A36110BD0268234643F814
:10291000102F53600022026022699A4203D1BDE861
:10292000104001F067BC936881680B44936001F02C
:1029300051FC2269E1699268441AA242E4D9114427
:10294000BDE81040091AFFF753BF00BF382D002023
:102950002DE9F047DFF8BC8008F110072C4ED8F8BD
:10296000105001F037FCD8F81C40AA68031B9A42AB
:102970003ED814444FF00009D5E90032C8F81C4095
:1029800013605A60C5F80090D8F81030B34201D1F6
:1029900001F030FC89F31188D5E9033128469847C6
:1029A000302383F311886B69002BD8D001F012FC1F
:1029B0006A69A0EB040982464A450DD2022001F063
:1029C00065FD0022D8F81030B34208D151462846A0
:1029D000BDE8F047FFF728BF121A2244F2E712EBD6
:1029E00009092946384638BF4A46FFF7EBFEB5E7E6
:1029F000D8F81030B34208D01444C8F81C00211A8B
:102A0000A960BDE8F047FFF7F3BEBDE8F08700BF5F
:102A1000482D0020382D002000207047FEE70000E0
:102A2000704700004FF0FF307047000002290CD0C3
:102A3000032904D00129074818BF00207047032A42
:102A400005D8054800EBC2007047044870470020D5
:102A5000704700BF084F000848220020BC4E000805
:102A600070B59AB005460846144601A900F0C2F8B0
:102A700001A8FEF7C9FA431C0022C6B25B0010464B
:102A8000C5E9003423700323023404F8013C01AB90
:102A9000D1B202348E4201D81AB070BD13F8011BB6
:102AA000013204F8010C04F8021CF1E708B53023E8
:102AB00083F311880348FFF725FA002383F3118875
:102AC00008BD00BFA82F002090F8803003F01F023F
:102AD000012A07D190F881200B2A03D10023C0E9F5
:102AE0001D3315E003F06003202B08D1B0F88430CB
:102AF0002BB990F88120212A03D81F2A04D8FFF788
:102B0000E3B9222AEBD0FAE7034A42670722826739
:102B1000C3670120704700BF3F22002007B5052989
:102B200017D8DFE801F0191603191920302383F3B1
:102B30001188104A01210190FFF78CFA01980221B7
:102B40000D4AFFF787FA0D48FFF7A8F9002383F332
:102B5000118803B05DF804FB302383F31188074824
:102B6000FFF772F9F2E7302383F311880348FFF788
:102B700089F9EBE75C4E0008804E0008A82F002082
:102B800038B50C4D0C4C2A460C4904F10800FFF7EF
:102B900067FF05F1CA0204F110000949FFF760FF61
:102BA00005F5CA7204F118000649BDE83840FFF780
:102BB00057BF00BF80480020482200203C4E00083C
:102BC000464E0008514E000870B5044608460D46B2
:102BD000FEF71AFAC6B22046013403780BB918463C
:102BE00070BD32462946FEF7FBF90028F3D10120DB
:102BF000F6E700002DE9F84F05460C46FEF704FA0B
:102C00002A49C6B22846FFF7DFFF08B10136F6B2FF
:102C100027492846FFF7D8FF08B11036F6B2632ED1
:102C20000DD8DFF88890DFF888A0224FDFF88CB04D
:102C3000DFF88C802E7846B92670BDE8F88F2946DB
:102C40002046BDE8F84F02F011B8252E2AD1072200
:102C500049462846FEF7C4F950B9D8F80030073580
:102C6000083444F8083CD8F8043044F8043CE1E760
:102C7000082251462846FEF7B3F998B9A21C0E4B1C
:102C8000197802320909C95D02F8041C13F8011B06
:102C900001F00F015B45C95D02F8031CF0D1183447
:102CA0000835C7E7013504F8016BC3E7284F000872
:102CB000514E0008394F000800E8F11F0CE8F11FE1
:102CC000304F0008BFF34F8F044B1A695107FCD1F6
:102CD000D3F810215207F8D1704700BF00200052EE
:102CE00008B50D4B1B78ABB9FFF7ECFF0B4BDA685F
:102CF000D10704D50A4A5A6002F188325A60D3F8E3
:102D00000C21D20706D5064AC3F8042102F1883205
:102D1000C3F8042108BD00BFDE4A00200020005295
:102D20002301674508B5114B1B78F3B9104B1A699D
:102D3000510703D5DA6842F04002DA60D3F8102177
:102D4000520705D5D3F80C2142F04002C3F80C21FC
:102D5000FFF7B8FF064BDA6842F00102DA60D3F8F9
:102D60000C2142F00102C3F80C2108BDDE4A00200C
:102D7000002000520F289ABF00F580604004002018
:102D8000704700004FF4003070470000102070477B
:102D90000F2808B50BD8FFF7EDFF00F500330268E8
:102DA000013204D104308342F9D1012008BD002052
:102DB000FCE700000F2838B505463FD8FFF782FF33
:102DC0001F4CFFF78DFF4FF0FF3307286361C4F8F6
:102DD00014311DD82361FFF775FF030243F024036C
:102DE000E360E36843F08003E36023695A07FCD49F
:102DF0002846FFF767FFFFF7BDFF4FF4003100F0F3
:102E0000C5F92846FFF78EFFBDE83840FFF7C0BF81
:102E1000C4F81031FFF756FFA0F108031B0243F07E
:102E20002403C4F80C31D4F80C3143F08003C4F807
:102E30000C31D4F810315B07FBD4D9E7002038BD42
:102E4000002000522DE9F84F04460D46104644EA92
:102E50000203DE0602D00020BDE8F88F20F01F003C
:102E6000DFF8D4B0DFF8D4A0FFF73AFF05EB000895
:102E7000454503D10120FFF755FFEDE72022294604
:102E8000204601F0E3FE10B920342035F0E7234658
:102E900004F120021F68791CDDD104339342F9D17B
:102EA00004F178432048214EB3F5801F204B38BFF2
:102EB000184603F1F80332BFD946D1461E46FFF744
:102EC00001FF0760A4EB050C336805F11C0143F01A
:102ED000020333602B1FD9F8007017F00507FAD1F1
:102EE00053F8042F8B424CF80320F4D1BFF34F8FDB
:102EF000FFF7E8FE4FF0FF330360336823F002036F
:102F00003360BFF34F8F0B4BC3F85C42BFF34F8F5F
:102F1000BFF36F8F20222946204601F097FE00283C
:102F2000B2D03846A7E700BF142100520C2000524F
:102F30001420005200ED00E0102000521021005239
:102F400010B5084C237828B11BB9FFF7C9FE01233F
:102F5000237010BD002BFCD02070BDE81040FFF79F
:102F6000E1BE00BFDE4A00202DE9F04F0D4685B0DE
:102F7000814658B111F00D0614BF2022082211F02D
:102F80000803019304D0431E03426AD0002435E0B5
:102F9000002E37D009F11F0121F01F094FF0010861
:102FA000324F05F00403DFF8D0A005EA080BBBF1AF
:102FB000000F32D07869C0072FD408F101080C3710
:102FC000B8F1060FF3D19EB9294D4946A8190192CF
:102FD00001F066F9044600283AD11836019A782E95
:102FE000F3D1494601F05CF90446002830D1019A3A
:102FF0004946204801F054F9044668BB204605B014
:10300000BDE8F08F0029C9D101462846029201F09F
:1030100047F90446E0B9029AC0E713B1786941075D
:10302000CBD5AC0702D578698007C6D5019911B117
:1030300078690107C1D51820494600FB08A0CDE9F1
:10304000022301F02DF90446DDE902230028B4D063
:103050004A460021204601E04A460021FDF7DCFFF8
:10306000CCE70246002E95D198E700BF4C4F0008F0
:10307000104B0020E04A0020F84A00200121FFF711
:1030800073BF0000F8B500231A461A600433B3F585
:10309000806FFAD1114D01241827114E07FB0460EF
:1030A00001342A6955F80C1F01F0E6F8062CF5D119
:1030B00037254FF4C0542046FFF7E0FF014628B102
:1030C00022460848BDE8F84001F0D6B8C4EBC40475
:1030D000013D4FEAD404EED1F8BD00BF4C4F0008CB
:1030E000F84A0020E04A002008B101F04BB97047CF
:1030F0000244074BD2B210B5904200D110BD441C1F
:1031000000B253F8200041F8040BE0B2F4E700BF2E
:10311000504000580E4B30B51C6F240405D41C6F72
:103120001C671C6F44F400441C670A4C024423686B
:10313000D2B243F480732360074B904200D130BD7C
:10314000441C51F8045B00B243F82050E0B2F4E7AD
:1031500000440258004802585040005807B5012268
:1031600001A90020FFF7C4FF019803B05DF804FB3C
:1031700013B50446FFF7F2FFA04205D0012201A9D2
:1031800000200194FFF7C6FF02B010BD0144BFF359
:103190004F8F064B884204D3BFF34F8FBFF36F8F1F
:1031A0007047C3F85C022030F4E700BF00ED00E098
:1031B000034B1A681AB9034AD2F8D0241A60704730
:1031C000884B00200040025808B5FFF7F1FF024B82
:1031D0001868C0F3806008BD884B0020EFF30983B6
:1031E000054968334A6B22F001024A6383F3098878
:1031F000002383F31188704700EF00E0302080F354
:10320000118862B60D4B0E4AD96821F4E0610904B9
:10321000090C0A430B49DA60D3F8FC2042F08072B3
:10322000C3F8FC20084AC2F8B01F116841F0010140
:1032300011602022DA7783F82200704700ED00E069
:103240000003FA0555CEACC5001000E0302310B5E0
:1032500083F311880E4B5B6813F4006314D0F1EE16
:10326000103AEFF309844FF08073683CE361094B37
:10327000DB6B236684F30988FFF7EAF910B1064B8C
:10328000A36110BD054BFBE783F31188F9E700BF8D
:1032900000ED00E000EF00E02F0400083204000819
:1032A00070B5BFF34F8FBFF36F8F1A4A0021C2F87A
:1032B0005012BFF34F8FBFF36F8F536943F4003346
:1032C0005361BFF34F8FBFF36F8FC2F88410BFF30A
:1032D0004F8FD2F8803043F6E074C3F3C900C3F3D4
:1032E0004E335B0103EA0406014646EA8175013963
:1032F000C2F86052F9D2203B13F1200FF2D1BFF394
:103300004F8F536943F480335361BFF34F8FBFF343
:103310006F8F70BD00ED00E0FEE70000214B2248FA
:10332000224A70B5904237D3214BC11EDA1C121AC3
:1033300022F003028B4238BF00220021FDF76CFE11
:103340001C4A0023C2F88430BFF34F8FD2F880307C
:1033500043F6E074C3F3C900C3F34E335B0103EAE1
:103360000406014646EA81750139C2F86C52F9D269
:10337000203B13F1200FF2D1BFF34F8FBFF36F8FBC
:10338000BFF34F8FBFF36F8F0023C2F85032BFF3EC
:103390004F8FBFF36F8F70BD53F8041B40F8041BB1
:1033A000C0E700BF785100087C4D00207C4D002014
:1033B0007C4D002000ED00E0074BD3F8D81021EA47
:1033C0000001C3F8D810D3F8002122EA0002C3F8A4
:1033D0000021D3F8003170470044025870B5D0E99D
:1033E000244300224FF0FF359E6804EB4213510145
:1033F000D3F80009002805DAD3F8000940F080402E
:10340000C3F80009D3F8000B002805DAD3F8000B45
:1034100040F08040C3F8000B013263189642C3F8B5
:103420000859C3F8085BE0D24FF00113C4F81C3808
:1034300070BD0000890141F02001016103699B0614
:10344000FCD41220FFF740B910B50A4C2046FEF715
:10345000DFFD094BC4F89030084BC4F89430084C99
:103460002046FEF7D5FD074BC4F89030064BC4F854
:10347000943010BD8C4B002000000840B84F00086D
:10348000284C002000000440C44F000870B50378A9
:103490000546012B5CD1434BD0F89040984258D15F
:1034A000414B0E216520D3F8D82042F00062C3F8CA
:1034B000D820D3F8002142F00062C3F80021D3F8ED
:1034C0000021D3F8802042F00062C3F88020D3F8B6
:1034D000802022F00062C3F88020D3F88030FEF70D
:1034E000FDF9324BE360324BC4F800380023D5F8C5
:1034F0009060C4F8003EC02323604FF40413A3631C
:103500003369002BFCDA01230C203361FFF7DCF870
:103510003369DB07FCD41220FFF7D6F83369002BA0
:10352000FCDA00262846A660FFF758FF6B68C4F84F
:103530001068DB68C4F81468C4F81C6883BB1D4BB2
:10354000A3614FF0FF336361A36843F00103A360FD
:1035500070BD194B9842C9D1134B4FF08060D3F81E
:10356000D82042F00072C3F8D820D3F8002142F0EE
:103570000072C3F80021D3F80021D3F8802042F074
:103580000072C3F88020D3F8802022F00072C3F8C4
:103590008020D3F88030FFF70FFF0E214D209EE7EB
:1035A000064BCDE78C4B00200044025840140040ED
:1035B00003002002003C30C0284C0020083C30C0F2
:1035C000F8B5D0F89040054600214FF0006620463F
:1035D000FFF730FFD5F8941000234FF001128F68E9
:1035E0004FF0FF30C4F83438C4F81C2804EB431201
:1035F00001339F42C2F80069C2F8006BC2F80809A3
:10360000C2F8080BF2D20B68D5F89020C5F89830B4
:10361000636210231361166916F01006FBD11220A5
:10362000FFF752F8D4F8003823F4FE63C4F80038EA
:10363000A36943F4402343F01003A3610923C4F8B2
:103640001038C4F814380B4BEB604FF0C043C4F88B
:10365000103B094BC4F8003BC4F81069C4F80039AA
:10366000D5F8983003F1100243F48013C5F8982080
:10367000A362F8BD944F000840800010D0F890205D
:1036800090F88A10D2F8003823F4FE6343EA01135D
:10369000C2F80038704700002DE9F84300EB8103C1
:1036A000D0F890500C468046DA680FFA81F948014C
:1036B000166806F00306731E022B05EB41134FF04C
:1036C000000194BFB604384EC3F8101B4FF001013F
:1036D00004F1100398BF06F1805601FA03F39169D3
:1036E00098BF06F5004600293AD0578A04F15801E0
:1036F000374349016F50D5F81C180B430021C5F81A
:103700001C382B180127C3F81019A7405369611EF4
:103710009BB3138A928B9B08012A88BF5343D8F826
:103720009820981842EA034301F140022146C8F864
:103730009800284605EB82025360FFF77BFE08EBFA
:103740008900C3681B8A43EA845348341E436401DA
:103750002E51D5F81C381F43C5F81C78BDE8F883F6
:1037600005EB4917D7F8001B21F40041C7F8001BEF
:10377000D5F81C1821EA0303C0E704F13F030B4A04
:103780002846214605EB83035A60FFF753FE05EBFD
:103790004910D0F8003923F40043C0F80039D5F8B7
:1037A0001C3823EA0707D7E7008000100004000256
:1037B000D0F894201268C0F89820FFF70FBE0000E0
:1037C0005831D0F8903049015B5813F4004004D0D0
:1037D00013F4001F0CBF0220012070474831D0F8BD
:1037E000903049015B5813F4004004D013F4001FDB
:1037F0000CBF02200120704700EB8101CB68196AE1
:103800000B6813604B6853607047000000EB810346
:1038100030B5DD68AA691368D36019B9402B84BF3D
:10382000402313606B8A1468D0F890201C4402EB8C
:103830004110013C09B2B4FBF3F46343033323F0BA
:10384000030343EAC44343F0C043C0F8103B2B6872
:1038500003F00303012B0ED1D2F8083802EB41101C
:1038600013F4807FD0F8003B14BF43F0805343F043
:103870000053C0F8003B02EB4112D2F8003B43F08A
:103880000443C2F8003B30BD2DE9F041D0F8906010
:1038900005460C4606EB4113D3F8087B3A07C3F8FC
:1038A000087B08D5D6F814381B0704D500EB810334
:1038B000DB685B689847FA071FD5D6F81438DB0732
:1038C0001BD505EB8403D968CCB98B69488A5A6843
:1038D000B2FBF0F600FB16228AB91868DA6890424B
:1038E0000DD2121AC3E90024302383F31188214634
:1038F0002846FFF78BFF84F31188BDE8F081012390
:1039000003FA04F26B8923EA02036B81CB68002B74
:10391000F3D021462846BDE8F041184700EB81036B
:103920004A0170B5DD68D0F890306C692668E660B1
:1039300056BB1A444FF40020C2F810092A6802F05E
:103940000302012A0AB20ED1D3F8080803EB42148D
:1039500010F4807FD4F8000914BF40F0805040F08C
:103960000050C4F8000903EB4212D2F8000940F0FD
:103970000440C2F800090122D3F8340802FA01F128
:103980000143C3F8341870BD19B9402E84BF4020DC
:10399000206020681A442E8A8419013CB4FBF6F496
:1039A00040EAC44040F00050C6E700002DE9F8436B
:1039B000D0F8906005460C464F0106EB4113D3F852
:1039C000088918F0010FC3F808891CD0D6F8103800
:1039D000DB0718D500EB8103D3F80CC0DCF81430FA
:1039E000D3F800E0DA68964530D2A2EB0E024FF031
:1039F00000091A60C3F80490302383F31188FFF79D
:103A00008DFF89F3118818F0800F1DD0D6F8343857
:103A10000126A640334217D005EB84030134D5F8C4
:103A20009050D3F80CC0E4B22F44DCF8142005EB1E
:103A30000434D2F800E05168714514D3D5F8343815
:103A400023EA0606C5F83468BDE8F883012303FAC3
:103A500001F2038923EA02030381DCF80830002B1A
:103A6000D1D09847CFE7AEEB0103BCF810008342FA
:103A700028BF0346D7F8180980B2B3EB800FE3D80C
:103A80009068A0F1040959F8048FC4F80080A0EBF5
:103A900009089844B8F1040FF5D818440B44906015
:103AA0005360C8E72DE9F84FD0F8905004466E698E
:103AB000AB691E4016F480586E6103D0BDE8F84F24
:103AC000FEF716BB002E12DAD5F8003E9B0705D094
:103AD000D5F8003E23F00303C5F8003ED5F80438BE
:103AE000204623F00103C5F80438FEF72FFB370505
:103AF00005D52046FFF772FC2046FEF715FBB00403
:103B00000CD5D5F8083813F0060FEB6823F4705382
:103B10000CBF43F4105343F4A053EB6031071BD5A3
:103B20006368DB681BB9AB6923F00803AB612378DA
:103B3000052B0CD1D5F8003E9A0705D0D5F8003EEC
:103B400023F00303C5F8003E2046FEF7FFFA636842
:103B5000DB680BB120469847F30200F1BA80B70248
:103B600026D5D4F8909000274FF0010A09EB4712B0
:103B7000D2F8003B03F44023B3F5802F11D1D2F8E3
:103B8000003B002B0DDA62890AFA07F322EA0303ED
:103B9000638104EB8703DB68DB6813B13946204699
:103BA00098470137D4F89430FFB29B689F42DDD923
:103BB000F00619D5D4F89000026AC2F30A1702F091
:103BC0000F0302F4F012B2F5802F00F0CA80B2F5B4
:103BD000402F09D104EB8303002200F58050DB68FD
:103BE0001B6A974240F0B0803003D5F8185835D59D
:103BF000E90303D500212046FFF746FEAA0303D5BB
:103C000001212046FFF740FE6B0303D50221204629
:103C1000FFF73AFE2F0303D503212046FFF734FEBA
:103C2000E80203D504212046FFF72EFEA90203D5A2
:103C300005212046FFF728FE6A0203D5062120460B
:103C4000FFF722FE2B0203D507212046FFF71CFEBB
:103C5000EF0103D508212046FFF716FE700340F15F
:103C6000A780E90703D500212046FFF79FFEAA079A
:103C700003D501212046FFF799FE6B0703D50221EA
:103C80002046FFF793FE2F0703D503212046FFF7B9
:103C90008DFEEE0603D504212046FFF787FEA80619
:103CA00003D505212046FFF781FE690603D50621CD
:103CB0002046FFF77BFE2A0603D507212046FFF7A3
:103CC00075FEEB0574D520460821BDE8F84FFFF7D7
:103CD0006DBED4F890904FF0000B4FF0010AD4F86D
:103CE00094305FFA8BF79B689F423FF638AF09EB41
:103CF0004713D3F8002902F44022B2F5802F20D1D7
:103D0000D3F80029002A1CDAD3F8002942F09042A7
:103D1000C3F80029D3F80029002AFBDB3946D4F880
:103D20009000FFF787FB22890AFA07F322EA0303D0
:103D3000238104EB8703DB689B6813B13946204677
:103D400098470BF1010BCAE7910701D1D0F8008029
:103D5000072A02F101029CBF03F8018B4FEA1828E1
:103D60003FE704EB830300F58050DA68D2F818C00F
:103D7000DCF80820DCE9001CA1EB0C0C00218F42D0
:103D800008D1DB689B699A683A449A605A683A4459
:103D90005A6029E711F0030F01D1D0F800808C455B
:103DA00001F1010184BF02F8018B4FEA1828E6E710
:103DB000BDE8F88F08B50348FFF774FEBDE808407A
:103DC000FFF744BA8C4B002008B50348FFF76AFEA2
:103DD000BDE80840FFF73ABA284C0020D0F89030F0
:103DE00003EB4111D1F8003B43F40013C1F8003B51
:103DF00070470000D0F8903003EB4111D1F8003942
:103E000043F40013C1F8003970470000D0F8903037
:103E100003EB4111D1F8003B23F40013C1F8003B40
:103E200070470000D0F8903003EB4111D1F8003911
:103E300023F40013C1F800397047000030B5043393
:103E4000039C0172002104FB0325C160C0E90653F5
:103E5000049B0363059BC0E90000C0E90422C0E99C
:103E60000842C0E90A11436330BD00000022416AE4
:103E7000C260C0E90411C0E90A226FF00101FEF737
:103E800093BC0000D0E90432934201D1C2680AB960
:103E9000181D704700207047036919600021C2682F
:103EA0000132C260C269134482699342036124BF34
:103EB000436A0361FEF76CBC38B504460D46E368FF
:103EC0003BB162690020131D1268A3621344E362D0
:103ED00007E0237A33B929462046FEF749FC00283B
:103EE000EDDA38BD6FF00100FBE70000C368C2697E
:103EF000013BC3604369134482699342436124BF19
:103F0000436A436100238362036B03B11847704720
:103F100070B53023044683F31188866A3EB9FFF7F3
:103F2000CBFF054618B186F31188284670BDA36AF9
:103F3000E26A13F8015B9342A36202D32046FFF7C3
:103F4000D5FF002383F31188EFE700002DE9F84F38
:103F500004460E46174698464FF0300989F31188FB
:103F60000025AA46D4F828B0BBF1000F09D141467C
:103F70002046FFF7A1FF20B18BF311882846BDE84A
:103F8000F88FD4E90A12A7EB050B521A934528BF04
:103F90009346BBF1400F1BD9334601F1400251F863
:103FA000040B914243F8040BF9D1A36A4036403523
:103FB0004033A362D4E90A239A4202D32046FFF792
:103FC00095FF8AF31188BD42D8D289F31188C9E7D9
:103FD00030465A46FCF7FAFFA36A5E445D445B44F0
:103FE000A362E7E710B5029C0433017203FB0421CE
:103FF000C460C0E906130023C0E90A33039B0363CE
:10400000049BC0E90000C0E90422C0E90842436300
:1040100010BD0000026A6FF00101C260426AC0E98F
:1040200004220022C0E90A22FEF7BEBBD0E9042325
:104030009A4201D1C26822B9184650F8043B0B607D
:10404000704700231846FAE7C3680021C2690133AC
:10405000C3604369134482699342436124BF436A46
:104060004361FEF795BB000038B504460D46E36892
:104070003BB1236900201A1DA262E2691344E36286
:1040800007E0237A33B929462046FEF771FB002862
:10409000EDDA38BD6FF00100FBE70000036919603D
:1040A000C268013AC260C2691344826993420361E3
:1040B00024BF436A036100238362036B03B1184783
:1040C0007047000070B530230D460446114683F357
:1040D0001188866A2EB9FFF7C7FF10B186F31188E1
:1040E00070BDA36A1D70A36AE26A01339342A362A2
:1040F00004D3E16920460439FFF7D0FF002080F3A4
:104100001188EDE72DE9F84F04460D469046994693
:104110004FF0300A8AF311880026B346A76A4FB9D8
:1041200049462046FFF7A0FF20B187F311883046AB
:10413000BDE8F88FD4E90A073A1AA8EB06079742B8
:1041400028BF1746402F1BD905F1400355F8042B13
:104150009D4240F8042BF9D1A36A40364033A36254
:10416000D4E90A239A4204D3E16920460439FFF7CF
:1041700095FF8BF311884645D9D28AF31188CDE794
:1041800029463A46FCF722FFA36A3D443E443B449D
:10419000A362E5E7D0E904239A4217D1C3689BB133
:1041A000836A8BB1043B9B1A0ED01360C368013B3A
:1041B000C360C3691A4483699A42026124BF436A97
:1041C0000361002383620123184670470023FBE745
:1041D00000F060BA014B586A704700BF000C004005
:1041E000034B002258631A610222DA60704700BF55
:1041F000000C0040014B0022DA607047000C0040C8
:10420000014B5863704700BF000C0040024B034A4B
:104210001A60034A5A607047DC4C0020804D002031
:1042200000000220074B494210B55C68201A084084
:104230001968821A8A4203D3A24201D85A6010BD7B
:104240000020FCE7DC4C002008B5302383F3118804
:10425000FFF7E8FF002383F3118808BD044801211C
:10426000044B03600023C0E901330C3000F016B9A1
:10427000E44C002049420008CB1D083A23F0070314
:10428000591A521A012110B4D2080024C0E900437F
:1042900084600C301C605A605DF8044B00F0FEB87E
:1042A0002DE9F84F364ECD1D0F46002818BF0646A3
:1042B000082A4FEAD50538BF082206F10C08341D3C
:1042C0009146404600F006F909F10701C9F1000ED8
:1042D000224624686CB9404600F006F93368CBB337
:1042E00008224946E8009847044698B340E9026727
:1042F00030E004EB010CD4F804A00CEA0E0C0AF137
:104300000100ACF1080304EBC0009842E0D9A0EB37
:104310000C0CB5EBEC0F4FEAEC0BD9D89C421CD23D
:1043200004F10802AB45A3EB02024FEAE20262602D
:1043300009D9691CED43206803EBC1025D44556057
:1043400043F8310022601C465F60404644F8086B29
:1043500000F0CAF82046BDE8F88FAA45216802D1CE
:1043600011602346EFE7013504EBC50344F835102F
:1043700003F10801401AC01058601360F1E700BF54
:10438000E44C0020F8B550F8043C044650F8085CB2
:10439000A0F1080607332F1D0C35DB0840F8043C5C
:1043A000284600F097F83B469F421A6801D0B34276
:1043B00028D20AB1964225D244F8082C54F8042C8D
:1043C0001E60013254F8081C06EBC200814206D17F
:1043D0004868024444F8042C0A6844F8082C5868D9
:1043E000411C03EBC1018E4207D154F8042C013269
:1043F00002445A6054F8082C1A602846BDE8F84078
:1044000000F072B81346CFE7FEE7000070B51B4B13
:104410000025044686B058600E4685620163FEF7AB
:10442000EDFE04F11003A560E562C4E904334FF02A
:10443000FF33C4E90044C4E90635FFF7CBFE2B4641
:10444000024604F134012046C4E9082380230C4AC3
:104450002565FEF743F901230A4AE06000920375DF
:10446000684672680192B268CDE90223064BCDE935
:104470000435FEF75BF906B070BD00BFA02F002029
:10448000D04F0008D54F000809440008024AD36AFB
:104490001843D062704700BF382D0020C0E90000EB
:1044A000816070478368013B002B10B583600CDA94
:1044B000074BDC684368A061206063601C60446057
:1044C0000520FEF77DF8A06910BD0020FCE700BFC5
:1044D000382D002008B5302383F31188FFF7E2FF61
:1044E000002383F3118808BD08B5302383F31188B6
:1044F00083680133002B836007DC036800211A689E
:10450000026050601846FEF787F8002383F3118895
:1045100008BD00004B6843608B688360CB68C36054
:104520000B6943614B6903628B6943620B680360EB
:104530007047000008B53C4B40F2FF713B48D3F890
:1045400088200A43C3F88820D3F8882022F4FF6229
:1045500022F00702C3F88820D3F88820D3F8E0209F
:104560000A43C3F8E020D3F808210A43C3F808211E
:104570002F4AD3F808311146FFF7CCFF00F58060D1
:1045800002F11C01FFF7C6FF00F5806002F138015F
:10459000FFF7C0FF00F5806002F15401FFF7BAFF9A
:1045A00000F5806002F17001FFF7B4FF00F5806054
:1045B00002F18C01FFF7AEFF00F5806002F1A80167
:1045C000FFF7A8FF00F5806002F1C401FFF7A2FF2A
:1045D00000F5806002F1E001FFF79CFF00F58060CC
:1045E00002F1FC01FFF796FF02F58C7100F5806087
:1045F000FFF790FF00F01AF90E4BD3F8902242F02B
:104600000102C3F89022D3F8942242F00102C3F8C9
:1046100094220522C3F898204FF06052C3F89C20E2
:10462000054AC3F8A02008BD004402580000025803
:10463000DC4F000800ED00E01F00080308B500F0A3
:10464000E5FAFEF725F8104BD3F8DC2042F04002E3
:10465000C3F8DC20D3F8042122F04002C3F804217F
:10466000D3F80431094B1A6842F008021A601A683C
:1046700042F004021A60FEF79BFDFEF703FDBDE861
:104680000840FEF77DBA00BF0044025800180248F7
:1046900070470000114BD3F8E82042F00802C3F83D
:1046A000E820D3F8102142F00802C3F810210C4A88
:1046B000D3F81031D36B43F00803D363C722094BFF
:1046C0009A624FF0FF32DA6200229A615A63DA602E
:1046D0005A6001225A611A60704700BF00440258B4
:1046E0000010005C000C0040094A08B51169D3684D
:1046F0000B40D9B29B076FEA0101116107D5302346
:1047000083F31188FDF7DEFF002383F3118808BDD2
:10471000000C0040064BD3F8DC200243C3F8DC2039
:10472000D3F804211043C3F80401D3F804317047CF
:104730000044025808B53C4B4FF0FF31D3F88020BD
:1047400062F00042C3F88020D3F8802002F00042DB
:10475000C3F88020D3F88020D3F88420C3F88410D5
:10476000D3F884200022C3F88420D3F88400D86FC3
:1047700040F0FF4040F4FF0040F4DF4040F07F0095
:10478000D867D86F20F0FF4020F4FF0020F4DF400E
:1047900020F07F00D867D86FD3F888006FEA4050C8
:1047A0006FEA5050C3F88800D3F88800C0F30A00BD
:1047B000C3F88800D3F88800D3F89000C3F89010AD
:1047C000D3F89000C3F89020D3F89000D3F8940069
:1047D000C3F89410D3F89400C3F89420D3F894004D
:1047E000D3F89800C3F89810D3F89800C3F898202D
:1047F000D3F89800D3F88C00C3F88C10D3F88C0051
:10480000C3F88C20D3F88C00D3F89C00C3F89C101C
:10481000D3F89C10C3F89C20D3F89C30FCF732FEF0
:10482000BDE8084000F0C2B90044025808B50122B2
:10483000534BC3F80821534BD3F8F42042F0020243
:10484000C3F8F420D3F81C2142F00202C3F81C2163
:104850000222D3F81C314C4BDA605A689104FCD523
:104860004A4A1A6001229A60494ADA6000221A61B3
:104870004FF440429A61444B9A699204FCD51A68FD
:1048800042F480721A603F4B1A6F12F4407F04D0DA
:104890004FF480321A6700221A671A6842F0010248
:1048A0001A60384B1A685007FCD500221A611A6941
:1048B00012F03802FBD1012119604FF0804159609C
:1048C0005A67344ADA62344A1A611A6842F480320A
:1048D0001A602C4B1A689103FCD51A6842F4805276
:1048E0001A601A689204FCD52C4A2D499A6200225B
:1048F0005A63196301F57C01DA6301F2E7119963E8
:104900005A64284A1A64284ADA621A6842F0A8529D
:104910001A601C4B1A6802F02852B2F1285FF9D1D4
:1049200048229A614FF48862DA6140221A621F4A73
:10493000DA641F4A1A651F4A5A651F4A9A6532236C
:104940001E4A1360136803F00F03022BFAD10D4ABD
:10495000136943F003031361136903F03803182B41
:10496000FAD14FF00050FFF7D5FE4FF08040FFF72F
:10497000D1FE4FF00040BDE80840FFF7CBBE00BFBE
:1049800000800051004402580048025800C000F066
:10499000020000010000FF010088900812102000B2
:1049A00063020901470E0508DD0BBF01200000204E
:1049B000000001100910E000000101100020005269
:1049C0004FF0B04208B5D2F8883003F00103C2F8C6
:1049D000883023B1044A13680BB150689847BDE88A
:1049E0000840FEF733BC00BFFC4C00204FF0B04243
:1049F00008B5D2F8883003F00203C2F8883023B13A
:104A0000044A93680BB1D0689847BDE80840FEF7A8
:104A10001DBC00BFFC4C00204FF0B04208B5D2F8DE
:104A2000883003F00403C2F8883023B1044A1369C4
:104A30000BB150699847BDE80840FEF707BC00BFBE
:104A4000FC4C00204FF0B04208B5D2F8883003F09B
:104A50000803C2F8883023B1044A93690BB1D069C6
:104A60009847BDE80840FEF7F1BB00BFFC4C0020B2
:104A70004FF0B04208B5D2F8883003F01003C2F806
:104A8000883023B1044A136A0BB1506A9847BDE8D5
:104A90000840FEF7DBBB00BFFC4C00204FF0B043EA
:104AA00010B5D3F8884004F47872C3F88820A306C0
:104AB00004D5124A936A0BB1D06A9847600604D5B0
:104AC0000E4A136B0BB1506B9847210604D50B4A65
:104AD000936B0BB1D06B9847E20504D5074A136C72
:104AE0000BB1506C9847A30504D5044A936C0BB1E5
:104AF000D06C9847BDE81040FEF7A8BBFC4C0020E6
:104B00004FF0B04310B5D3F8884004F47C42C3F8AA
:104B10008820620504D5164A136D0BB1506D984775
:104B2000230504D5124A936D0BB1D06D9847E0046C
:104B300004D50F4A136E0BB1506E9847A10404D5EB
:104B40000B4A936E0BB1D06E9847620404D5084AA5
:104B5000136F0BB1506F9847230404D5044A936F29
:104B60000BB1D06F9847BDE81040FEF76FBB00BF98
:104B7000FC4C002008B50348FCF72AFEBDE80840BD
:104B8000FEF764BB5C24002008B50348FCF720FE58
:104B9000BDE80840FEF75ABBC824002008B5FFF75F
:104BA000A3FDBDE80840FEF751BB0000062108B593
:104BB0000846FCF793FE06210720FCF78FFE06212E
:104BC0000820FCF78BFE06210920FCF787FE062152
:104BD0000A20FCF783FE06211720FCF77FFE062142
:104BE0002820FCF77BFE09217A20FCF777FE0721BD
:104BF0003220FCF773FE0C212520FCF76FFE0C2100
:104C00003420BDE80840FCF769BE000008B5FFF796
:104C100091FD00F00DF8FDF71FF8FDF7F7F9FDF72E
:104C2000C9F8FFF735FDBDE80840FFF7D1BA00002D
:104C30000023054A19460133102BC2E9001102F185
:104C40000802F8D1704700BFFC4C002010B50139B4
:104C50000244904201D1002005E0037811F8014F91
:104C6000A34201D0181B10BD0130F2E7034611F832
:104C7000012B03F8012B002AF9D1704753544D330F
:104C80003248373F3F3F0053544D33324837337833
:104C90002F3732780053544D3332483734332F375F
:104CA00035332F373530000001105A0003105900FA
:104CB0000120580003205600100002400800024066
:104CC0000008024000000B002800024008000240DB
:104CD0000408024006010C004000024008000240A7
:104CE0000808024010020D0058000240080002406F
:104CF0000C08024016030E00700002400C00024037
:104D00001008024000040F00880002400C0002401E
:104D10001408024006051000A00002400C000240EA
:104D20001808024010061100B80002400C000240B2
:104D30001C08024016072F0010040240080402401D
:104D400020080240000838002804024008040240FD
:104D500024080240060939004004024008040240C9
:104D600028080240100A3A00580402400804024091
:104D70002C080240160B3B00700402400C04024059
:104D800030080240000C3C00880402400C04024041
:104D900034080240060D4400A00402400C04024006
:104DA00038080240100E4500B80402400C040240CE
:104DB0003C080240160F460000960000000000006C
:104DC00000000000000000000000000000000000E3
:104DD00000000000191C0008051C0008411C000808
:104DE0002D1C0008391C0008251C0008111C000897
:104DF000FD1B00084D1C000800000000311D0008CC
:104E00001D1D0008591D0008451D0008511D000802
:104E10003D1D0008291D0008151D0008651D00081E
:104E200000000000010000000000000063300000EE
:104E30002C4E0008902D0020A02F00204172647598
:104E400050696C6F740025424F415244252D424CED
:104E5000002553455249414C250000000200000046
:104E600000000000511F0008C11F00084000400062
:104E700050480020604800200200000000000000B0
:104E800003000000000000000920000800000000EE
:104E90001000000070480020000000000100000029
:104EA000000000008C4B0020010102001D2B0008B7
:104EB0002D2A0008C92A0008AD2A00084300000076
:104EC000C44E000809024300020100C03209040078
:104ED0000001020201000524001001052401000167
:104EE000042402020524060001070582030800FFCE
:104EF00009040100020A0000000705010240000049
:104F0000070581024000000012000000104F000859
:104F10001201100102000040091241570002010273
:104F2000030100000403090425424F4152442500B7
:104F3000414544524F5848370030313233343536CA
:104F40003738394142434445460000000000002004
:104F50000000020002000000000000300000040019
:104F60000800000000000024000008000400000009
:104F70000004000000FC00000200000000000430FB
:104F80000080000008000000000000380000010060
:104F90000100000000000000652100081D24000839
:104FA000C924000840004000C44C0020C44C00202C
:104FB00001000000D44C00208000000040010000EF
:104FC00008000000000100000010000008000000C0
:104FD0006D61696E0069646C650000000001A86A7B
:104FE00000000000AAAAAAAA00011464FFFF0000A2
:104FF0000000000070A70A00000000000000000090
:10500000AAAAAAAA00000000FFFF000000000000FA
:10501000000000000000000000000000AAAAAAAAE8
:1050200000000000FFFF0000000000000000000082
:105030000A00000000000000AAAAAAAA05000000B9
:10504000FFFF0000880000000000000000050000D5
:1050500000000000AAAAAAAA00000000FFFF0000AA
:105060000000000000000000000000000000000040
:10507000AAAAAAAA00000000FFFF0000000000008A
:10508000000000000000000000000000AAAAAAAA78
:1050900000000000FFFF0000000000000000000012
:1050A0000000000000000000AAAAAAAA0000000058
:1050B000FFFF0000000000000000000000000000F2
:1050C00000000000AAAAAAAA00000000FFFF00003A
:1050D00000000000000000000000000000000000D0
:1050E000AAAAAAAA00000000FFFF0000000000001A
:1050F000000000000000000000000000AAAAAAAA08
:1051000000000000FFFF00000000000000000000A1
:10511000AE0400000000000000001A0000000000C3
:10512000FF000000A82F00205C240020C8240020DD
:10513000000000007C4C000883040000874C00083D
:1051400050040000954C0008009600000000080084
:10515000960000000008000004000000244F000832
:10516000000000000000000000000000000000003F
:08517000000000000000000037
:00000001FF
